:0400000010EF00F00D
:08000800FACF7FFF57EF0DF066
:10001800D8CF64FF51EF0DF00AEE21F01FEE64F027
:10002800BEEC24F000EE11F010EE13F0BEEC24F05C
:1000380000EE77F011EE00F0BEEC24F0FAEF0DF0D0
:100048000001CF6BD06BD16BD26B2C0ED36F0A0E25
:10005800D46FDDEC1BF0006E00C002F0036A0350A1
:100068000210D8B4000CEECBE8FF040AD8B405D0CF
:10007800EECBE8FF060AD8A40AD02ACCE8FF550A36
:10008800D8A405D02BCCE8FFAA0AD8B406D0000122
:10009800856B866B876B886B44D0F2CB00F00001D0
:1000A80000C085F0866B876B886B080EF3CB00F079
:1000B800016A026A036A92EC24F000EE85F00050AF
:1000C800EE260150EE220250EE220350ED22ED52B0
:1000D800ED52100EFECB00F0016A026A036A92EC40
:1000E80024F000EE85F00050EE260150EE2202507A
:1000F800EE220350ED22ED52ED52180EFFCB00F028
:10010800016A026A036A92EC24F000EE85F000505E
:10011800EE260150EE220250EE220350ED22ED525F
:10012800ED5285C0CFF086C0D0F087C0D1F088C02E
:10013800D2F000012C0ED36F0A0ED46FDDEC1BF049
:10014800006E00C002F0036A03500210D8B4000C1D
:100158002CCAE8FFE90AD8B405D02CCAE8FFEB0A94
:10016800D8A4000C0AEE37F0EF50D8A4000C38CA17
:10017800E8FF020AD8A4000C41CAE8FFF80AD8A48C
:10018800000C3ECA7CF03DCA7BF07BC000F07CC00E
:1001980001F0050ED89000360136E82EFBD7000690
:1001A800010E0122090E026ED89001320032022E91
:1001B800FBD700500001BA6F0150BB6FBC6BBD6B21
:1001C8003BCA01F0006A000E01BEFF0E026E036E0C
:1001D8003ACAE8FF0024046E000E0120056E000EE6
:1001E8000220066E000E0320076E00EE85F0045014
:1001F800EE260550EE220650EE220750ED22ED5273
:10020800ED5243CA01F0006A42CAE8FF0024046EB6
:10021800000E0120056E066A05BE06060650076E2A
:1002280004C0BEF005C0BFF006C0C0F007C0C1F0F2
:100238003CCA2BFABEC004F0BFC005F0C0C006F02F
:10024800C1C007F02BCA00F0016A026A036AE0EC39
:1002580023F085C0E8FF0024E8CF81F086C0E8FFDE
:100268000120E8CF82F087C0E8FF0220E8CF83F0C2
:1002780088C0E8FF0320E8CF84F039CA2AFABA0E0A
:10028800E96E000EEA6E0001EE508125E8CF7DF0A0
:10029800EE508221E8CF7EF0EE508321E8CF7FF048
:1002A800ED508421E8CF80F0ED52ED52010CBE00F4
:1002B8000001C36BC46BC56BC66BBEC0D9FFBFC0A2
:1002C800DAFFC051D8A409D000EE0CF0D950E926C5
:1002D800DA50EA22EE6AED6AC9D10001C005D8B445
:1002E800BCD10001C051020AD8A4C0D1ACD181C090
:1002F80004F082C005F083C006F084C007F000EE69
:100308000CF0D950E926DA50EA22EECF00F0EDCF12
:1003180001F0040E026ED89001320032022EFBD793
:10032800026A036A00500426015005220250062280
:100338000350072200EE0CF0D950E926DA50EA22E1
:10034800EECF00F0EDCF01F00F0E0016000E0116F3
:10035800050ED89000360136E82EFBD700C0C1F054
:1003680001C0C2F0D9CFBEF0DACFBFF0000107500C
:10037800C61908E10650C51905E10550C41902E17E
:100388000450C319D8B41ED004C0C3F005C0C4F0CB
:1003980006C0C5F007C0C6F0C3C0CFF0C4C0D0F0D7
:1003A800C5C0D1F0C6C0D2F02C0ED36F0A0ED46FE0
:1003B800DDEC1BF0006E00C002F0036A035002106F
:1003C800D8B4000CBEC0D9FFBFC0DAFF00010AEEE6
:1003D8002CF0C151E926C251EA22EF50D8B42ED1EF
:1003E8000AEE2CF0C151E926C251EA22EF50E50A83
:0803F800D8B424D100010AEE83
:100400002CF0C151E926C251EA22EF502E0AD8B48D
:1004100019D100010AEE37F0C151E926C251EA2292
:10042000EF501A0BD8A40ED1F36AF3500001C12586
:10043000006E000EC221016E2C0E0024E16E0A0E29
:100440000120E26EF350D924E96E000EDA20EA6E44
:10045000E7CFEFFFF32A0A0EF364E7D7F350D9246E
:10046000E96E000EDA20EA6EEF6AF3500AEE48F009
:10047000E926000EEA22EF50006E00C002F0036A87
:1004800000EE10F0D950E926DA50EA2202C0EEFF61
:1004900003C0EDFF0AEE49F0C151E926C251EA223C
:1004A000EF50016E006A00EE10F0D950E926DA50E4
:1004B000EA220050EE260150ED2200EE10F0D95055
:1004C000E926DA50EA22EE06010EED22090E006E50
:1004D00000EE10F0D950E926DA50EA22002804D0C4
:1004E000D890EC32ED52EF32E82EFAD70AEE4AF00D
:1004F000C151E926C251EA22EF50006E00C002F05D
:10050000036A070ED89002360336E82EFBD700EEBA
:1005100010F0D950E926DA50EA220250EE260350B4
:10052000ED220AEE46F0C151E926C251EA22EF500F
:10053000006E0AEE47F0C151E926C251EA22EF509F
:10054000036E00C002F000EE16F0D950E926DA5032
:10055000EA2202C0EEFF03C0EDFF0AEE4BF0C151EC
:10056000E926C251EA22EF50006E016A026A036A6C
:10057000080E92EC24F000C0C7F001C0C8F002C021
:10058000C9F003C0CAF00AEE4AF0C151E926C251CF
:10059000EA22EF50006E016A026A036AC751002620
:1005A000C8510122C9510222CA510322080E92ECFD
:1005B00024F000C0CBF001C0CCF002C0CDF003C0ED
:1005C000CEF00AEE49F0C151E926C251EA22EF50BD
:1005D000006E016A026A036ACB510026CC510122E7
:1005E000CD510222CE510322080E92EC24F00AEEE5
:1005F00048F0C151E926C251EA22EF500024046EAE
:10060000000E0120056E000E0220066E000E032073
:10061000076E00EE12F0D950E926DA50EA2204C043
:10062000EEFF05C0EEFF06C0EEFF07C0EDFFED5286
:10063000ED5200EE0EF0D950E926DA50EA22EE6AC9
:10064000ED6A010C0001C051020AD8A40AD000EEE4
:100650000CF0D950E926DA50EA22EE06000EED5AE7
:1006600009D000EE0CF0D950E926DA50EA22EE2A41
:10067000000EED227BC000F07CC001F000EE0CF01B
:10068000D950E926DA50EA22EECF02F0EDCF03F09E
:100690000150035C02E10050025CD8A02CD600EEB1
:1006A00010F0D950E926DA50EA22EE6AED6A000C21
:1006B000BA000001BC6BBD6B000100EE16F0BA5130
:1006C000E926BB51EA22D890BC35006EBD35016EDB
:1006D0002C0E0024E16E0C0E0120E26EEECFE6FF40
:1006E000EDCFE5FFBAC0C7F0BBC0C8F021D8006E9F
:1006F00000C002F0036A03500210D8B4000C0001DD
:10070000BC4BBD2B010EBD5D7F0ED8B4BC5DD8A027
:10071000D3D7000110EE16F0BA51E126BB51E22208
:100720000FEE2AF0E6CFEEFFE5CFEDFF010CC7009C
:10073000C7C0E1FFC8C0E2FF00EE0EF0E150E926BD
:10074000E250EA22EE2A000EED222ACA02F0036AE3
:1007500000EE0EF0E150E926E250EA22EECF00F082
:10076000EDCF01F023EC24F001500010D8A4010CCF
:1007700085C0CBF086C0CCF087C0CDF088C0CEF06D
:1007800000EE16F0E150E926E250EA22EECF00F04A
:10079000EDCF01F001C000F0016A026A036A0001B6
:1007A0000050CB270150CC230250CD230350CE2341
:1007B00000EE16F0E150E926E250EA22EECF00F01A
:1007C000EDCF01F00050C96FCA6BE1CFC7F0E2CFA7
:1007D000C8F0D890C937CA37CBC0CFF0CCC0D0F062
:1007E000CDC0D1F0CEC0D2F02C0ED36F0A0ED46F94
:1007F000DDEC1BF0006E00C002F0036A0350021033
:10080000D8B4000C00010AEE2CF0C951E926CA51F7
:10081000EA22EF50006E0AEE2DF0C951E926CA51C6
:10082000EA22EF50036E00C002F000EE16F0C7514E
:10083000E926C851EA2202C0EEFF03C0EDFF010C19
:10084000D000090ED2C000F0D3C001F0D4C002F035
:10085000D5C003F0A8EC24F000C0E4F001C0E5F03E
:1008600002C0E6F003C0E7F00001D251DC6F010ED8
:10087000D315DD6FDE6BDF6BD0C0D9FFD1C0DAFFDF
:10088000D651DC25006ED751DD21016E000EDE2130
:10089000026E000EDF21036E000E035C08E1000E05
:1008A000025C05E1020E015C02E1000E005CD8B0C2
:1008B0000BD0D651E06FD751E16FE26BE36BD86B91
:1008C000D96BDA6BDB6B25D0DC0EE96E000EEA6EBD
:1008D0000001EE500008E06F020EEE54E16F000ED2
:1008E000EE54E26F000EED54E36FED52ED52D6C0C0
:1008F00000F0D7C001F0026A036AE051005CD86FD3
:10090000E1510158D96FE2510258DA6FE3510358AF
:10091000DB6F0001D890E435006EE535016E2C0EDA
:100920000024E16E0C0E0120E26E00EE16F0D950AC
:10093000E926DA50EA22E6CFEEFFE5CFEDFF00EE42
:100940000EF0D950E926DA50EA22E4C0EEFFE5C005
:10095000EDFF7DC0E8F07EC0E9F07FC0EAF080C026
:10096000EBF02ACA02F0036A00EE16F0D950E9262D
:10097000DA50EA22EECF00F0EDCF01F0FE0E0026B5
:10098000FF0E0120016E84EC24F004C000F005C0CD
:1009900001F0026A036A0050E8270150E92302507F
:1009A000EA230350EB232ACA02F0036A00EE0EF09A
:1009B000D950E926DA50EA22EECF00F0EDCF01F06F
:1009C00023EC24F0026A036A0050E8270150E9236F
:1009D0000250EA230350EB23D9CFD0F0DACFD1F085
:1009E000E8C0ECF0E9C0EDF0EAC0EEF0EBC0EFF0EB
:1009F000DCC0F0F0DDC0F1F02C0EF26F0A0EF36FE8
:100A0000E0C0F4F0E1C0F5F071EC1BF0006E00C046
:100A100002F0036A03500210D8B4000C0001DB514D
:100A2000D811D911DA11D8B4010CD890E435006E80
:100A3000E535016E2E0E0024E16E0C0E0120E26EF3
:100A400000EE16F0D051E926D151EA22E6CFEEFFB2
:100A5000E5CFEDFFD0C0E1FFD1C0E2FFE4C000F080
:100A6000E5C001F0E6C002F0E7C003F0002A000E86
:100A7000012200EE0EF0E150E926E250EA2200C029
:100A8000EEFF01C0EDFF7DC0E8F07EC0E9F07FC061
:100A9000EAF080C0EBF02ACA02F0036A00EE16F01A
:100AA000E150E926E250EA22EECF00F0EDCF01F06E
:100AB000FE0E0026FF0E0120016E84EC24F004C01F
:100AC00000F005C001F0026A036A0050E8270150F7
:100AD000E9230250EA230350EB232ACA02F0036AF7
:100AE00000EE0EF0E150E926E250EA22EECF00F0EF
:100AF000EDCF01F023EC24F0026A036A0050E827EE
:100B00000150E9230250EA230350EB23E8C0ECF044
:100B1000E9C0EDF0EAC0EEF0EBC0EFF0F06BF16B86
:100B20002D0EE025F26F0A0EE121F36FD8C0F4F02C
:100B3000D9C0F5F071EC1BF0006E00C002F0036A42
:100B400003500210D8B4000C010CC7007DC0C9F0DE
:100B50007EC0CAF07FC0CBF080C0CCF0C7C0E1FF40
:100B6000C8C0E2FF2ACA02F0036A00EE16F0E150A4
:100B7000E926E250EA22EECF00F0EDCF01F0FE0EC2
:100B80000026FF0E0120016E84EC24F004C000F06A
:100B900005C001F0026A036A00010050C927015034
:100BA000CA230250CB230350CC232ACA02F0036A83
:100BB00000EE0EF0E150E926E250EA22EECF00F01E
:100BC000EDCF01F023EC24F0026A036A0050C9273C
:100BD0000150CA230250CB230350CC23C9C0CFF00D
:100BE000CAC0D0F0CBC0D1F0CCC0D2F02C0ED36FA5
:100BF0000A0ED46FDDEC1BF0006E00C002F0036A39
:100C000003500210D8B4000C010C0001BA6FB9D91E
:100C1000BFD9C4D911941198BAC063FF1200B1D9D9
:100C2000B7D9BCD981A0FED781A01200FDD70001A1
:100C3000BF6F11941198C16B080EC06F80A4FED7CE
:100C4000ADD90001880EC26F130EC36F000EC46FC2
:100C5000C56F000180A44BD0C207000EC35BC45B0C
:100C6000C55BC551C211C311C411D8A4F2D71184F8
:100C700098D9460E0001CE6FCF6BD5EC22F08ED9FD
:100C8000E8D70001D890C133C007880E006E130E5C
:100C9000016E000E026E036E80A4FED70006000EE9
:100CA000015A025A035A0350001001100210D8A42E
:100CB00002D01188000C80A603D0800E0001C1274D
:100CC000880E006E130E016E000E026E036E80B46D
:100CD000FED70006000E015A025A035A03500010B4
:100CE00001100210D8A402D01188000C0001C051DC
:100CF000D8A4C7D70001BF51D8A406D0E20ECE6F4A
:100D0000040ECF6FD5EC22F04CD90001C151120076
:100D10000001CC6F080ECD6F11983AD980A6FED78E
:100D200011A432D0C80E0001CE6FCF6BD5EC22F0EB
:100D3000880E006E130E016E000E026E036E80B6FA
:100D4000FED70006000E015A025A035A0350001043
:100D500001100210D8A402D01188000C880E006E79
:100D6000130E016E000E026E036E80A6FED7000603
:100D7000000E015A025A035A0350001001100210CB
:100D8000D8A402D01188000C06D9500E0001CE6FF5
:100D9000CF6BD5EC22F00001CD51D8B418D0FBD8E0
:100DA000500E0001CE6FCF6BD5EC22F00001CD07C5
:100DB000CCA102D0F3D801D0F4D8EAD80001D89061
:100DC000CC33500ECE6FCF6BD5EC22F0E4D7E3D806
:100DD000E5D8880E006E130E016E000E026E036ED3
:100DE00080B6FED70006000E015A025A035A03507D
:100DF000001001100210D8A402D01188000C640E5B
:100E00000001CE6FCF6BD5EC22F0010CC9000001C0
:100E1000CB6B0001CB51C925006E000ECA21016EBB
:100E200000C0F6FF01C0F7FF0F0EF76403D0080003
:100E3000F55005D0F6CFE9FFF7CFEAFFEF500009F4
:100E4000D8B412000001CB51C925006E000ECA2192
:100E5000016E00C0F6FF01C0F7FF0F0EF76403D06C
:100E60000800F55005D0F6CFE9FFF7CFEAFFEF50C5
:100E70004FDF0001CB2BCDD7D96E0A0E016ED950B2
:100E800056EC24F0300F0001BB6FD950BA6FBB5144
:100E90003FDF0A0E016E0001BA5156EC24F00050FB
:100EA000300FBB6FBB5134D780A4FED777D83C0E30
:100EB0000001CE6FCF6BD5EC22F06DD83C0E000157
:100EC000CE6FCF6BD5EC22F0010C6BD83C0E00013D
:100ED000CE6FCF6BD5EC22F05BD83C0E0001CE6F0D
:100EE000CF6BD5EC22F080A4010CFDD7000CBA002A
:100EF000C80E0001CE6FCF6BD5EC22F081A002D0DE
:100F00004DD8FCD74ED80001BC5191DEBAC0E9FFE4
:100F1000BBC0EAFFEF6EBAC0E1FFBBC0E2FFE75023
:100F20000F0BD96E11A881B0E3D7E750006E63CFE5
:100F3000E8FF20090018D8B4200CE7503F0AD8B4C5
:100F40003F0CE750006E63CFE8FF40090018D8B4AB
:100F5000400CE7505F0AD8B45F0CE750F00BF00A82
:100F6000D8B4F00CE750F00BE00AD8B4E00CE7502E
:100F7000F00B600AD8A4BCD7D9500F0AD8B46F0CB4
:100F8000600C8180938012009350936E81901200C8
:100F900080849284120092948094120080869286BB
:100FA0001200929680961200066A01AE06D0001ECC
:100FB000004A0106011E068C068E0350800B061A9D
:100FC00003AE24EF24F0021E024A0306031E24EFA0
:100FD00024F0036A026A016A006AE950EA1008E034
:100FE00003C0EDFF02C0EDFF01C0EDFF00C0EFFF49
:020FF000000CF3
:1010000000151515151515151515151515151515A5
:1010100015151313131313131312121212121211A4
:10102000111111111111111111043314332433242E
:1010300033243324332433243324332433243324F8
:1010400033243324332433243324332433243324E8
:101050003334333433343334333433443354333428
:10106000334433643374337433743374337433A458
:1010700034A434A434A4347433A434A434A434A4E1
:1010800034A434A434A434A434A434A434843394D1
:1010900033A433A434A434A434A434A434A434A492
:1010A00034B433C433D433E433F433043414342445
:1010B00034A434A434343444345434643494347D07
:1010C00060606060606060606060606060607D0063
:1010D0007D53454C2E20443634203A243F3F3F7DFB
:1010E000007D20313534312D49494920284A442991
:1010F0007D007D53454C2E20434152443A243020FC
:10110000207D007D4449524543544F52593A242092
:1011100020207D00726F6F74206469726563746F44
:10112000727900313534312D4949492076002573D3
:10113000006A606060606060606060606060606005
:101140006B007560606060606060606060606060DF
:101150006069000D0D313534312D4949492076251E
:10116000642E25642C206279204A2E4465726F67B4
:1011700065650046696C653A2020253033642F256B
:101180003033640025633D2530326420543D2530E2
:10119000326420533D253032640044524956452084
:1011A0004E4F54205245414459005245434F5244FA
:1011B000204E4F542050524553454E540046494C02
:1011C000452045584953545300494C4C4547414CE0
:1011D0002053595354454D2054204F522053004919
:1011E0004C4C4547414C20545241434B20414E44C6
:1011F00020534543544F52004449524543544F52A3
:1012000059204552524F520053594E54415820458F
:1012100052524F52005752495445204552524F5254
:101220000052454144204552524F52004552524FC0
:101230005220554E4B4F4E574E0057524954452061
:1012400050524F54454354204F4E0046494C452080
:101250004E4F54204F50454E00575249544520465A
:10126000494C45204F50454E004449534B2046556C
:101270004C4C004E4F204348414E4E454C004F4B86
:10128000004E4F20424C4F434B0046494C452054A2
:10129000595045204D49534D41544348004449530A
:1012A0004B204944204D49534D4154434800464941
:1012B0004C4520544F4F204C41524745004F564516
:1012C00052464C4F5720494E205245434F524400FE
:1012D00046494C45204E4F5420464F554E440046FB
:1012E000494C455320534352415443484544004ED2
:1012F0002F4100533A00433A00403A0053303A003D
:1013000043303A0040303A0043617264206E6F749B
:1013100020737570702E0045723A256420622E622B
:101320006C2E00284A2E4445524F4745452900243B
:101330000045723A766F6C74206572726F7221008C
:1013400045723A434D443538206661696C21004549
:10135000723A696E69742E206661696C210043617E
:101360007264206465746563746564200020434181
:101370005244204449524543544F52592000496E2B
:1013800069742E20636172643A20202000424C4F21
:10139000434B5320465245452E202020202020201C
:1013A00020202020202020200000FE81FE0000FEC2
:1013B000C1FE0000FEE1FE0000FEF1FE0000FEF9AD
:1013C000FE0000FEFDFE0000FEFFFE00181FC1F83B
:1013D0000818423C817E0000000000000000000070
:1013E00000000000000000000000FA00F090FE3E47
:1013F0003E363E3E384444282800FE7C38101038E3
:101400007CFE000C0A000C0A0A06000A0688CCEED4
:10141000CC882266EE6622387C7C7C382070A8203E
:101420003E0804FE04082040FE40201010543810EE
:101430001038541010808894A28080A29488804034
:10144000707C7040041C7C1C040000000000000044
:10145000BE0000000E000E0028FE28FE284854FEA4
:101460005424462610C8C46C92AA44A000000A0660
:10147000000038448200008244380028107C102884
:1014800010107C101000A060000010101010100050
:10149000C0C0000040201008047CA2928A7C008416
:1014A000FE800084C2A2928C42828A9662302824F6
:1014B000FE204E8A8A8A7278949292600602E21224
:1014C0000E6C9292926C0C9292523C00CCCC00002A
:1014D00000AC6C000010284482002828282828002E
:1014E000824428100402A2120C6492F2827CF82436
:1014F0002224F8FE9292926C7C82828244FE828246
:101500004438FE92929282FE121212027C829292D1
:10151000F4FE101010FE0082FE82004080827E02E7
:10152000FE10284482FE80808080FE041804FEFEA7
:10153000081020FE7C8282827CFE1212120C7C82B9
:10154000A242BCFE1232528C4C929292640202FE73
:1015500002027E8080807E3E4080403EFE403040E1
:10156000FEC6281028C60E10E0100EC2A2928A866F
:1015700000FE8282000408102040008282FE0008E3
:10158000040204088080808080000204080040A8D3
:10159000A8A8F0FE90888870708888884070888835
:1015A00090FE70A8A8A83010FC12020410A8A8A8E9
:1015B00078FE100808F00090FA80004080887A00D9
:1015C00000FE2050880082FE8000F808F008F8F83D
:1015D000100808F07088888870F8282828100814E7
:1015E0001418FCF81008081090A8A8A840087E88D5
:1015F000804078808040F838408040387880608033
:1016000078885020508818A0A0A07888C8A898880A
:1016100000106C82000000FE000000826C100010C0
:1016200008081008F0888488F0000000000000001E
:1016300000000000000000000000000000000000AA
:10164000000000000000000000000000000000009A
:10165000000000000000000000000000000000008A
:10166000000000000000000000000000000000007A
:10167000000000000000000000000000000000006A
:10168000000000000000000000000000000000005A
:10169000000000000000000000000000000000004A
:1016A000000000000000000000000000000000003A
:1016B000000000000000000000000000000000002A
:1016C000000000000000000000000000000000001A
:1016D000000000000000000000000000000000000A
:1016E00000000000000000000000000000000000FA
:1016F00000000000000000000000000000000000EA
:1017000000000000000000000000000000000000D9
:1017100000000000000000000000000000000000C9
:1017200000000000000000000000000000000000B9
:1017300000000000000000000000000000000000A9
:101740000000000000000000000000000000000099
:101750000000000000000000000000000000000089
:101760000000000000000000000000000000000079
:101770000000000000000000000000000000000069
:101780000000000000000000000000000000000059
:101790000000000000000000000000000000000049
:1017A0000000000000000000000000000000000039
:1017B0000000000000000000000000000000000029
:1017C0000000000000000000000000000000000019
:1017D0000000000000000000000000000000000009
:1017E00000000000000000000000000000000000F9
:1017F00000000000000000000000000000000000E9
:101800000000000000000000001C222E221C1C22F0
:101810002A261C1C222A2A1C1C222A321C1C223A80
:10182000221C1C322A221C1C2A2A221C1C262A2288
:101830001C0000000000000000000000000000008C
:101840000000000000000000000000000000000098
:10185000000000000000000000C3A79FA7C3C3A5AD
:101860009FA7C3C3A59FA5C3C3A5BFA5C3C3A5BD4C
:10187000A5C3C3A5FDA5C3C3E5FDA5C3C3E5F9E5A0
:10188000C300000000000000000000000000000095
:101890000000000000000000000000000000000048
:1018A00000000000000000000000E020A0A0A02038
:1018B000A0A0A020A0A04080000000000000000028
:1018C000FCFC04048404F4946404F4A4E404744468
:1018D000F4440404FCFC00000010F01000F0501070
:1018E00000E01010000000000000000000000000F8
:1018F0008080808080800000000000000000FF00E9
:1019000043300B005B6803784B320000FF0020205F
:10191000A8702000FEFFFEFEFEFEFEFEFECE8686C6
:1019200086CEFEFEFEFEFEFEFFFE0070887101F90F
:1019300000F901F90070897100F8002020A87020DA
:1019400000F8FEFF8F070303070707D8D8D8D88809
:1019500000001F101E101E101E101E101E101E1044
:101960001F000000000000007F7F7F7F7F7F7F7F60
:101970007F7F7F437F7F7F7F7F7F7F7F7F7F0000B1
:101980000000000000000000000000000000000057
:1019900000000000000003070F0F0E0E0F0F0700DE
:1019A000000000000000D0D0D0D0D0D0D0D0D0D017
:1019B000D0D0D0D0D0D0D0D0D0D000E0B010F00077
:1019C000F010D05050700080E010F0000000E0B047
:1019D00010F0000000000070D010D050D010D05097
:1019E000D010D0700000D0D0D0D0D0D0D0D0D0D0B7
:1019F000D0D0D0D0D0D0D0D0D0D0EEEEEEEEEEEE33
:101A0000EEEEEEEEEEEEEEEEEEEEEEEEEEEE0000D2
:101A1000FF80FF007794A5BD837E003F202FE984DF
:101A2000EC1800FF80FF000E0A0A0EE0BF80BFA086
:101A3000BF80BFA0BF80BFE00000EEEEEEEEEEEE96
:101A4000EEEEEEEEEEEEEEEEEEEEEEEEEEEEFDFD98
:101A5000FDFDFDFDFDFDFDFDFDFDFDFDFDFDFDFDB6
:101A6000FDFD00007C50200C503C00000020403C5C
:101A70000040007C4438007C54007C1468003844EA
:101A8000380038445434007C54007C540000FDFD80
:101A9000FDFDFDFDFDFDFDFDFDFDFDFDFDFDFDFD76
:021AA000FD0047
:101AA2009EB09E9064CFD8FF1000FAD7E9CF7EFF98
:101AB200EACF7DFFE1CF7CFFE2CF7BFFD9CF7AFF78
:101AC200DACF79FF0EC078FF0DC077FF0CC076FF2A
:101AD2000BC075FF0AC074FF09C073FF08C072FF14
:101AE20007C071FF06C070FF05C06FFF04C06EFF24
:101AF20003C06DFF02C06CFF01C06BFF00C06AFF34
:101B0200F7CF69FFF6CF68FFF5CF67FFF4CF66FF27
:101B1200F3CF65FFF2A203D0F292D1EC07F0F2A468
:101B220031D0D59EF2942CCFE8FF030AD8A420D05E
:101B320011A604D011962DCFD6FF05D011862DCF38
:101B4200E8FF0008D66ED7682DCF00F00004D8B4A5
:101B520011822DCFE8FFFE0AD8B4119211A204D04F
:101B62000F01010E2D2B08D00F01010E2D0704D0FD
:101B72001176F60ED76ED66A11A602D0808201D0F7
:101B82008092D58E65CFF3FF66CFF4FF67CFF5FF66
:101B920068CFF6FF69CFF7FF6ACF00F06BCF01F095
:101BA2006CCF02F06DCF03F06ECF04F06FCF05F073
:101BB20070CF06F071CF07F072CF08F073CF09F043
:101BC20074CF0AF075CF0BF076CF0CF077CF0DF013
:101BD20078CF0EF079CFDAFF7ACFD9FF7BCFE2FF51
:101BE2007CCFE1FF7DCFEAFF7ECFE9FF7FCFFAFF17
:0E1BF20011000001D00EBA6F070EBB6F14EC8D
:101C000023F094EC23F0080EE8CF33FF33CFE8FF46
:101C100005EC06F0118017EC21F00001530EDF6F88
:101C2000110EE06FB86BB96B010EB66FB76BB60EE5
:101C3000E8CFDDF0000EE8CFDEF09DEC24F0010EE1
:101C40000001C96F490E47EC19F0020E2EEC23F08B
:101C5000D3DA51EC12F0030E0001C96F490E47ECC4
:101C600019F02DEC21F00001BA6BBB6B7CDB00019D
:101C7000C96BCA6BCB6BCC6BCD6B000EDEDB00018E
:101C8000AB6BAA6B00018D6B8E6BC80E0001CE6F23
:101C9000CF6BD5EC22F00001310EBA6F0F0EBB6F87
:101CA000010EBC6F78EC07F00001A76FC80ECE6F75
:101CB000CF6BD5EC22F00001A751200AD8B404D094
:101CC000A751400AD8A404D0010E0001AA6FDDD7A5
:101CD0000001AA51D8A4E7D10FEC06F0D6D70FEC3B
:101CE00006F0DED10FEC06F0DBD100013A0EBA6F40
:101CF0000F0EBB6F010EBC6FBD6BEAD9320E000137
:101D0000BA6FBB6B14EC23F000012F0EBA6F130EE9
:101D1000BB6F3A0EBC6F0F0EBD6F010EBE6FBF6B77
:101D200067EC22F0015000100001D8A480D03B0ED7
:101D3000BA6F0F0EBB6FB20EBC6F000EBD6FEBD94A
:101D4000006E00C002F0036A03500210D8B466D0DF
:101D50000001B551B211B311B411D8A404D00001DF
:101D60008D6B8E6B60D0020E0001AB6FB2C08DF038
:101D7000B3C08EF0AE6BAF6BB06BB16B8DC000F0CB
:101D80008EC001F0026A036A00010350B15D08E1F0
:101D90000250B05D05E10150AF5D02E10050AE5D63
:101DA000D8B034D00001B151AE11AF11B011D8A4E8
:101DB00008D08F0EBE6F000EBF6FC06B5CEC01F0E1
:101DC0001ED000018F0EBE6F000EBF6F010EC06FE0
:101DD0005CEC01F0006E00C002F0036A03500210D8
:101DE000D8A40DD0020E0001C96F150E47EC19F0F2
:101DF00000018D6B8E6B0A0E0001AB6F07D00001E6
:101E0000AE2B000EAF23B023B123B8D700018F0E45
:101E1000BA6F000EBB6F59EC03F037D700018D513C
:101E20008E11D8A402D0010EACD0020EAAD0F90EA9
:101E3000BA6F120EBB6F3A0EBC6F0F0EBD6F020E63
:101E4000BE6FBF6B67EC22F001500010D8B412D007
:101E50000001040EBA6F130EBB6F3A0EBC6F0F0E6B
:101E6000BD6F030EBE6FBF6B67EC22F00150001018
:101E7000D8A402D0050E85D00001F30EBA6F120E61
:101E8000BB6F3A0EBC6F0F0EBD6F020EBE6FBF6B05
:101E900067EC22F001500010D8B412D00001FC0E03
:101EA000BA6F120EBB6F3A0EBC6F0F0EBD6F030EF2
:101EB000BE6FBF6B67EC22F001500010D8A402D0B7
:101EC000070E5FD00001F60EBA6F120EBB6F3A0E0E
:101ED000BC6F0F0EBD6F020EBE6FBF6B67EC22F0C2
:101EE00001500010D8B4C6D70001000EBA6F130E0F
:101EF000BB6F3A0EBC6F0F0EBD6F030EBE6FBF6B94
:101F000067EC22F001500010D8B4B4D700018D5115
:101F10008E1100013A0ED8A41AD0BA6F0F0EBB6F03
:101F20008F0EBC6F000EBD6F9FEC17F0006E00C0EF
:101F300002F0036A03500210D8B402D0040E21D07C
:101F4000020E0001C96F3E0E47EC19F023D0BA6FA4
:101F50000F0EBB6FA90EBC6F000EBD6FA80EBE6F3B
:101F6000000EBF6FAC0EC06F000EC16FA4EC1FF06F
:101F7000006E00C002F0036A03500210D8B404D00F
:101F8000030E0001AB6F81D6020E0001C96F3E0E39
:101F900047EC19F00A0EF5D778D65FD00FEC06F0B3
:101FA00074D654EC07F00FEC06F06FD6D7EC13F0B4
:101FB0006CD68DC0BAF08EC0BBF0D5D98DC000F004
:101FC0008EC001F000500001BA6F0150BB6FBC6BB6
:101FD000BD6BA6EC15F059D6020E0001D76F000EAE
:101FE00061EC21F000012E0EDF6F110EE06F3A0E52
:101FF000B86F0F0EB96FB80EE8CFDDF0000EE8CF66
:10200000DEF09DEC24F000018F0EBA6F000EBB6F66
:1020100023EC18F03AD6020E0001D76F000E61ECE7
:1020200021F000012E0EDF6F110EE06F3A0EB86F37
:102030000F0EB96FB80EE8CFDDF0000EE8CFDEF07E
:102040009DEC24F00001A851BA6FACC0BBF0ADC04C
:10205000BCF0A951C8EC18F018D60001AB519EE0B5
:10206000010AA4E0030AA5E0010AD5E0070AB4E0EA
:10207000010AF2E0030AF0E0010AEEE00F0AECE0E8
:10208000010AEAE0030A8DE000D676EC19F0FDD5EE
:102090000FEC06F0020E0001C96F1E0E47EC19F09E
:1020A0000001AA6BF2D50001A7513F0A01E117D642
:1020B000600A01E117D63F0A01E16FD70F0AE5E098
:1020C0008F0A01E169D7100A01E10FD6E1D7BA0002
:1020D000119811940001BE6B0FD00001BC5117EC98
:1020E00006F0006E0001BE51BA25E96E000EBB215C
:1020F000EA6E00C0EFFFBE2B11B802D011A4EDD7DD
:102100000001BE51BA25E96E000EBB21EA6E000E39
:10211000EF6A1200BA00E16ABCC0D9FFBDC0DAFFA5
:10212000D9CFE9FFDACFEAFFEE6AEE6AEE6AED6A2E
:1021300046D00A0E046E056A066A076AD9CFE9FF1F
:10214000DACFEAFFEECF00F0EECF01F0EECF02F0F3
:10215000EECF03F0E0EC23F000C0DEFF01C0DEFFB5
:1021600002C0DEFF03C0DDFFDD52DD52E1500001A1
:10217000BA25E96E000EBB21EA6EEF50006E016ACF
:10218000D00E0026FF0E0122026A036ADE500024F0
:10219000046EDE500120056EDE500220066EDD501A
:1021A0000320076EDD52DD5204C0DEFF05C0DEFFF6
:1021B00006C0DEFF07C0DDFFDD52DD52E12AE1503F
:1021C0000001BA25E96E000EBB21EA6EEF50006EE9
:1021D000300E005CD8A00CD0E150BA25E96E000E9C
:1021E000BB21EA6EEF50006E3A0E005CD8A0A1D77A
:1021F000E150D8B4000C010C010E0001D76F000EA5
:1022000061EC21F000019A0EDF6F130EE06F9DEC80
:1022100024F0020E0001D76F000E61EC21F00001E6
:102220009A0EDF6F130EE06F9DEC24F00001D76B68
:10223000000E61EC21F000015E0EDF6F130EE06F07
:102240009DEC24F0020E2EEC23F00001D76B000E63
:1022500061EC21F000017E0EDF6F130EE06F9DEC4C
:1022600024F0010E0001D76F000E61EC21F025D89B
:102270000009D8B41ED024EC00F00009D8A40DD079
:102280000001D76B000E61EC21F00001080EDF6F3A
:10229000130EE06F9DEC24F00CD00001D76B0B0EF9
:1022A00061EC21F000017E0EDF6F120EE06F9DEFFA
:1022B00024F0030E2EEC23F0B9D78CEC1AF00009B1
:1022C0000001D8A407D04F0EDF6F130EE06F9DEC16
:1022D00024F0000C350EBC6F0F0EBD6F28EC1BF008
:1022E000006E00C002F0036A03500210D8A408D0A8
:1022F0000001400EDF6F130EE06F9DEC24F0000C28
:1023000037CFE8FF3C0B3C0AD8B408D00001310EAF
:10231000DF6F130EE06F9DEC24F0000C0001896B61
:10232000020E8A6F89C0BCF08AC0BDF062EC1BF05F
:10233000006E00C002F0036A03500210D8A4010C22
:102340000001170EDF6F130EE06F89C0BAF08AC06C
:10235000BBF0BA0EE8CFDDF0000EE8CFDEF09DEC6A
:1023600024F0000CBA000001D76B000E61EC21F0E4
:102370000001730EDF6F110EE06F8BC0BEF08CC0DA
:10238000BFF0BAC0BCF0BBC0BDF0BC0EE8CFDDF002
:10239000000EE8CFDEF09DEC24F0010E0001D76FB7
:1023A000000E61EC21F00001BB51BA11D8A40BD092
:1023B00094EC21F00001140EDF6F110EE06F9DEC24
:1023C00024F096EF21F094EC21F0200EC0EC23F0E5
:1023D0008FC0E8FFC0EC23F090C0E8FFC0EC23F012
:1023E00091C0E8FFC0EC23F092C0E8FFC0EC23F0FE
:1023F00093C0E8FFC0EC23F094C0E8FFC0EC23F0EA
:1024000095C0E8FFC0EC23F096C0E8FFC0EC23F0D5
:102410002E0EC0EC23F097C0E8FFC0EC23F098C06C
:10242000E8FFC0EC23F099C0E8FFC0EC23F0200ED9
:10243000C0EC23F096EF21F0C9000001CE6F040E2E
:10244000D76F000E61EC21F00001CC51D76FCA515B
:1024500033EC22F0050E0001D76F000E61EC21F085
:102460000001840EDF6F110EE06FC9C000F0016A39
:1024700000C0D5F001C0D6F0CEC000F0016A00C0A7
:10248000D3F001C0D4F033CFD1F0D26B0D0ECF6FAB
:10249000D06BCF0EE8CFDDF0000EE8CFDEF09DEF81
:1024A00024F000018F0EBE6F000EBF6FC06B5CEC9E
:1024B00001F0006E00C002F0036A03500210000138
:1024C000D8B44BD0010E8B6F8C6B00018F0EBE6F9A
:1024D000000EBF6F010EC06F5CEC01F0006E00C01B
:1024E00002F0036A03500210D8B42FD00001A151AA
:1024F000AB0ED8B4A219020ED8B4A319D8B4A45103
:10250000D8A40FD097C0E8FF440AD8A40AD098C036
:10251000E8FF360AD8A405D099C0E8FF340AD8B439
:102520000FD097C0E8FF500AD8A4CFD798C0E8FFD3
:10253000520AD8A4CAD799C0E8FF470AD8A4C5D779
:1025400000018B2B000E8C23C0D700018F0EBE6FB5
:10255000000EBF6FC06B5CEF01F08B6B8C6B1200D9
:102560008DC0A7F08EC0A8F06CD811AC2AD00001A5
:10257000A851A711D8B419D0A705A811D8B412D062
:1025800000018F0EBE6F000EBF6F020EC06F5CECBD
:1025900001F0006E00C002F0036A03500210D8B4CC
:1025A00004D00001A707D8A0A807A7C0BAF0A8C008
:1025B000BBF0D9DE00015E0EBA6F010EBB6F14ECEA
:1025C00023F011AA30D08BC000F08CC001F00001C4
:1025D0000150A85D02E10050A75DD8B018D0A85105
:1025E000A711D8B412D000018F0EBE6F000EBF6FBE
:1025F000010EC06F5CEC01F0006E00C002F0036AD7
:1026000003500210D8B403D00001A74BA82BA7C0D9
:10261000BAF0A8C0BBF0A7DE00015E0EBA6F010ED3
:10262000BB6F14EC23F011AE9FD7A7C08DF0A8C0EC
:102630008EF000018F0EBA6F000EBB6F59EC03F0E5
:1026400093D70001A76BA86BA96BAA6B810EC26E12
:10265000C282C2B2FED7C450016E006AC3500024C9
:10266000026E000E0120036E02C004F003C005F0EC
:10267000000E05BEFF0E066E076E0001AA1908E1E6
:10268000A951061805E1A851051802E1A75104183F
:10269000D8B40ED004C0A7F005C0A8F006C0A9F0B9
:1026A00007C0AAF0810EC26EC282C2A2D4D7FDD7E3
:1026B000F80E0426FD0E0522FF0E06220722119CAD
:1026C000119E119A520E0424006EFF0E0520016E19
:1026D000FF0E0620026EFF0E0720036E0350800AD5
:1026E000810F08E1FF0E025C05E1FF0E015C02E1D3
:1026F000F60E005CD8A007D0520E0426FF0E05226D
:1027000006220722118CB40E0424006EFF0E052051
:10271000016EFF0E0620026EFF0E0720036E0350AF
:10272000800A810F08E1FF0E025C05E1FF0E015CEB
:1027300002E1F60E005CD8A007D0B40E0426FF0E0E
:10274000052206220722118EDF0E0424006EFF0EE2
:102750000520016EFF0E0620026EFF0E0720036E9D
:102760000350800A810F08E1FF0E025C05E1FF0EB5
:10277000015C02E1F60E005CD8A007D0DF0E042653
:10278000FF0E052206220722118A0750800A800FB9
:1027900008E1000E065C05E1000E055C02E11A0E80
:1027A000045CD8A01200119C119E119A1200010E17
:1027B0000001C96F000E47EC19F0119454EC07F0BA
:1027C000010E88EC06F0040E88EC06F0010E88EC91
:1027D00006F0010E88EC06F0000E88EC06F0000E04
:1027E00088EC06F0200E88EC06F0120E88EC06F05D
:1027F000220E88EC06F000016D0EC96F130ECA6F31
:1028000007EC07F0220E88EC06F0000E88EC06F0CC
:10281000010E88EC06F0010E88EC06F0000E88EC44
:1028200006F0000E88EC06F0200E88EC06F0220E72
:1028300088EC06F00001420EC96F110ECA6F07EC5A
:1028400007F0220E88EC06F0000E88EC06F0010E70
:1028500088EC06F0010E88EC06F0000E88EC06F01D
:10286000000E88EC06F0200E88EC06F0220E88ECB4
:1028700006F00001E10EC96F100ECA6F07EC07F0F9
:10288000220E88EC06F0000E88EC06F0010E88ECB3
:1028900006F0010E88EC06F0000E88EC06F0000E43
:1028A00088EC06F0200E88EC06F0220E88EC06F08C
:1028B0000001BF0EC96F100ECA6F07EC07F0220EA1
:1028C00088EC06F0000E88EC06F0010E88EC06F0AD
:1028D000010E88EC06F0000E88EC06F0000E88EC85
:1028E00006F0200E88EC06F0220E88EC06F00001BF
:1028F000030EC96F110ECA6F07EC07F0220E88ECA9
:1029000006F0000E88EC06F0010E88EC06F0010ED1
:1029100088EC06F0000E88EC06F0000E88EC06F05D
:10292000200E88EC06F0220E88EC06F00001F20E74
:10293000C96F100ECA6F07EC07F0220E88EC06F084
:10294000000E88EC06F0010E88EC06F0010E88EC13
:1029500006F0000E88EC06F0000E88EC06F0200E63
:1029600088EC06F0220E88EC06F00001D00EC96F4C
:10297000100ECA6F07EC07F0220E88EC06F0000E6E
:1029800088EC06F0010E88EC06F0010E88EC06F0EB
:10299000000E88EC06F0000E88EC06F0200E88ECA5
:1029A00006F0220E88EC06F00001310EC96F110E00
:1029B000CA6F07EC07F0220E88EC06F0000E88ECD8
:1029C00006F00001BA6B8F0EBE6F000EBF6FC06BBA
:1029D0005CEC01F0006E00C002F0036A03500210CC
:1029E000D8B4A6D00001BA2B0001A151AB0ED8B4C7
:1029F000A219020ED8B4A319D8B4A451D8A40FD0E8
:102A000097C0E8FF440AD8A40AD098C0E8FF360A65
:102A1000D8A405D099C0E8FF340AD8B40FD097C025
:102A2000E8FF500AD8A473D098C0E8FF520AD8A48F
:102A30006ED099C0E8FF470AD8A469D0010E88EC8F
:102A400006F0010E88EC06F00001BA5188EC06F0A1
:102A5000026A010E036EBAC000F0016AD4EC07F0FE
:102A6000045088EC06F00A0E0001BA6103D0200E73
:102A700088EC06F0220E88EC06F08FC0E8FF88ECA8
:102A800006F090C0E8FF88EC06F091C0E8FF88EC03
:102A900006F092C0E8FF88EC06F093C0E8FF88ECEF
:102AA00006F094C0E8FF88EC06F095C0E8FF88ECDB
:102AB00006F096C0E8FF88EC06F02E0E88EC06F0D3
:102AC00097C0E8FF88EC06F098C0E8FF88EC06F0B5
:102AD00099C0E8FF88EC06F0220E88EC06F0000EA4
:102AE00088EC06F00001C96BBA518BC000F08CC0B5
:102AF00001F0005CCA6F0150D8A00104CB6F00EE5A
:102B0000CCF08BC0EEFF8CC0EDFF000E96DC000118
:102B10008F0EBE6F000EBF6F010EC06F5CEC01F038
:102B2000006E00C002F0036A03500210D8A45AD706
:102B3000000E88EC06F01184000E88EC06F065ECBF
:102B400007F0030E0001C96F9FD3BA00010E000108
:102B5000C96F000E9CDB119454EC07F0010E88EC59
:102B600006F0040E88EC06F000018F0EC96F000E0F
:102B7000CA6F120ECB6FCC6B900ECD6F190ECE6F4D
:102B8000CF6BC1EC20F0010E0001C76FC86BC96BA1
:102B9000010ECA6FCB6BCC6BCD6B120E4EDC010EEF
:102BA00088EC06F0010E88EC06F00001BA5188ECC2
:102BB00006F00001BB5188EC06F0120E88EC06F01E
:102BC000220E88EC06F00001C16B0001C1510AEE33
:102BD0002CF0E926000EEA22EF5088EC06F0000106
:102BE000C12B0F0EC165F1D7220E88EC06F0200E26
:102BF00088EC06F03ECAE8FF88EC06F03FCAE8FF22
:102C000088EC06F0200E88EC06F041CAE8FF88EC5C
:102C100006F042CAE8FF88EC06F0000E88EC06F0E9
:102C20000001BE6B0001BE514EEC1FF00009D8B48C
:102C30005ED10001C74BC82B2ECFC9F0C7C0CAF068
:102C4000C8C0CBF0CC6BCD6B2FCFE8FF1DEC12F0E2
:102C5000010E0001BE6FBF6B45D10001BF39E846D0
:102C6000E00B020FC26FC2510AEE2CF0E926000EF3
:102C7000EA22EF50D8B434D1010E88EC06F0010EF0
:102C800088EC06F00001C2510AEE48F0E926000E79
:102C9000EA22EF5088EC06F00001C2510AEE49F03A
:102CA000E926000EEA22EF5088EC06F00001C2513E
:102CB0000AEE48F0E926000EEA22EF50006EC251FB
:102CC0000AEE49F0E926000EEA22EF50C66F00C076
:102CD000C5F0000EC65D0A0ED8B4C55DD8B003D0ED
:102CE000200E88EC06F00001000EC65D640ED8B41C
:102CF000C55DD8B003D0200E88EC06F00001030EAD
:102D0000C65DE80ED8B4C55DD8B003D0200E88ECFF
:102D100006F0220E88EC06F00001C06B030EC16FB6
:102D20000001C251C1C000F0016A0026000E01225C
:102D30002C0E0024E96E0A0E0120EA6EEF50A00A64
:102D4000D8B411D0C251C1C000F0016A0026000EF3
:102D500001222C0E0024E96E0A0E0120EA6EEF50CB
:102D6000200AD8A408D00001C02B1AD0200E88EC6D
:102D700006F00001C0070001C051D8A4F7D7000138
:102D8000C251C1C000F0016A0026000E01222C0EC3
:102D90000024E96E0A0E0120EA6EEF5088EC06F07E
:102DA0000001C12B120EC165BBD7220E88EC06F0C4
:102DB0000001C051D8B406D0200E88EC06F0000106
:102DC000C007F6D70001C2510AEE2CF0E926000E2A
:102DD000EA22EF50006E400E0016410E005CD8A0B3
:102DE00004D03E0E88EC06F047D00001C2510AEE36
:102DF0002CF0E926000EEA22EF50006E800E005CF7
:102E0000D8A004D0200E88EC06F036D02A0E88EC2C
:102E100006F032D0440E88EC06F0450E88EC06F041
:102E20004C0E88EC06F04DD0530E88EC06F0450EA3
:102E300088EC06F0510E88EC06F043D0500E88EC7A
:102E400006F0520E88EC06F0470E88EC06F039D0FA
:102E5000550E88EC06F0530E88EC06F0520E88EC06
:102E600006F02FD0520E88EC06F0450E88EC06F0E6
:102E70004C0E88EC06F025D00001C2510AEE2CF071
:102E8000E926000EEA22EF50006E070E001600C081
:102E900002F0036A0BD00250BDE0010AC5E0030A4C
:102EA000CDE0010AD5E0070ADDE002D00350F3E0EF
:102EB000550E88EC06F04E0E88EC06F04B0E88ECB2
:102EC00006F0200E88EC06F0200E88EC06F0200EAE
:102ED00088EC06F0200E88EC06F0000E88EC06F078
:102EE0000001BF2B070E0001BF65B7D69BD6010EB0
:102EF00088EC06F0010E88EC06F078EC1FF000C0BC
:102F0000C3F001C0C4F00001C35188EC06F0000119
:102F1000C45188EC06F000018D0EC96F130ECA6F04
:102F200007EC07F0000E88EC06F0000E88EC06F0C7
:102F30001184000E88EC06F065EC07F0A3D1BCC04C
:102F4000BEF0BDC0BFF00001C06B5CEC01F0006ED4
:102F500000C002F0036A03500210D8B4000CD96814
:102F6000D92ABCC0E1FFBDC0E2FFD950080AD8A4ED
:102F70001ED000EE08F0E150E926E250EA22EF50C0
:102F8000500AD8A414D000EE09F0E150E926E2502E
:102F9000EA22EF50520AD8A40AD000EE0AF0E1501B
:102FA000E926E250EA22EF50470AD8B4010C0001AA
:102FB000BA51D924E96E000ED9BEFF0EBB21EA6ECC
:102FC000EF50D8B436D00001BA51D924E96E000EC2
:102FD000D9BEFF0EBB21EA6EEF503F0AD8A408D03D
:102FE000D950E124E96E000EE220EA6E3F0EEF6E4A
:102FF0000001BA51D924E96E000ED9BEFF0EBB21E3
:10300000EA6EEF502A0AD8B4010CBA51D924E96EFD
:10301000000ED9BEFF0EBB21EA6EEF50006ED950F4
:10302000E124E96E000EE220EA6EEF500018D8B4F9
:1030300097D7BCC0BEF0BDC0BFF0010E0001C06F8D
:103040005CEC01F084D7010E0001C96F000E1FD99E
:10305000119454EC07F0BAC0E1FFBBC0E2FF00EEF0
:1030600012F0E150E926E250EA22EECFC3F0EECFB3
:10307000C4F0EECFC5F0EECFC6F00001BF6BC06B61
:10308000BC6BFE0E046E056A066A076AC3C000F0D8
:10309000C4C001F0C5C002F0C6C003F039EC23F093
:1030A00000C0C1F001C0C2F0C1C0BDF0C2C0BEF0DE
:1030B000FE0E046E056A066A076AC3C000F0C4C04B
:1030C00001F0C5C002F0C6C003F039EC23F0075090
:1030D000041005100610D8B402D0C14BC22B000159
:1030E000C107D8A0C207E1CFC7F0E2CFC8F0A6EC75
:1030F00005F00001C651C311C411C511D8B444D0A4
:103100000001C305C411C511C611D8B411840AEE5B
:103110002CF0BF51E926C051EA22EF5088EC06F0AE
:103120000001C307000EC45BC55BC65BBC2BBF4B75
:10313000C02BC051020ABF11D8A40FD0BAC0C7F02B
:10314000BBC0C8F098EC03F0BAC0C7F0BBC0C8F071
:10315000A6EC05F00001BF6BC06B0001BC51FE0A7C
:10316000D8A4C7D7C107D8A0C207C96BC1C0CAF0CD
:10317000C2C0CBF0BDC0CCF0BEC0CDF0000E1DEC87
:1031800012F00001BC6BB5D765EC07F0DAD4BA00D9
:103190000001BD6FBBC0BFF0BCC0C0F0010EC96F65
:1031A000000E75D8119454EC07F00001BD51D8B44D
:1031B00037D000018F0EC96F000ECA6FBD51CB6FA3
:1031C000BA51CC6FCD6BCE6B010ECF6FC1EC20F03E
:1031D0002CCABDF02DCABAF00001BF07D8A0C007A5
:1031E000BA51C96FBFC0CAF0C0C0CBF0BBC0CCF0F1
:1031F000BCC0CDF0BD511DEC12F0020E0001BE6F3F
:103200000001BE510AEE2CF0E926000EEA22EF5032
:1032100088EC06F00001BE2BBE51D8B4C6D7F0D75B
:10322000020E0001BE6F0001FF0EBA25026E036A96
:10323000FF0E0322BEC000F0016A0150800A046E36
:103240000350800A045C02E10250005CD8B00DD04B
:103250000001BE510AEE2CF0E926000EEA22EF50E2
:1032600088EC06F00001BE2BDED711840001BA51B4
:103270000AEE2CF0E926000EEA22EF5088EC06F068
:1032800065EC07F00001C96B000E01D0C900D96ED2
:10329000D950D8B421D034CFE8FF490AD8A4D9CF27
:1032A00034FF1AD0D59E80921200D59E80821200E3
:1032B000020EE8CF2CFF1196D768D668D58E120083
:1032C000030EE8CF2CFF11921196D768D668D58EE1
:1032D0001200D59E809212000001C951E3E0010A5C
:1032E000E4E0030AE5E0010AEBE0F3D71194808201
:1032F00054EC07F034CFE8FF3CEC07F02C0E88ECE0
:1033000006F0D8D000017E0EC96F120ECA6F07EC0E
:1033100007F0E4D00001DF0EC96F120ECA6F07EC90
:1033200007F0DCD00001EF0EC96F120ECA6F07EC78
:1033300007F0D4D00001210EC96F120ECA6F07EC3E
:1033400007F0CCD00001150EC96F120ECA6F07EC42
:1033500007F0C4D000013A0EC96F120ECA6F07EC15
:1033600007F0BCD000019D0EC96F120ECA6F07ECAA
:1033700007F0B4D00001080EC96F120ECA6F07EC37
:1033800007F0ACD00001AA0EC96F110ECA6F07EC8E
:1033900007F0A4D00001BD0EC96F120ECA6F07EC72
:1033A00007F09CD00001AE0EC96F120ECA6F07EC79
:1033B00007F094D00001590EC96F120ECA6F07ECC6
:1033C00007F08CD000014B0EC96F120ECA6F07ECCC
:1033D00007F084D00001D00EC96F120ECA6F07EC3F
:1033E00007F07CD00001BD0EC96F110ECA6F07EC4B
:1033F00007F074D000018A0EC96F120ECA6F07EC75
:1034000007F06CD00001810EC96F120ECA6F07EC75
:1034100007F064D00001DF0EC96F110ECA6F07EC10
:1034200007F05CD00001C90EC96F110ECA6F07EC1E
:1034300007F054D00001730EC96F120ECA6F07EC6B
:1034400007F04CD00001F80EC96F110ECA6F07ECDF
:1034500007F044D00001690EC96F120ECA6F07EC65
:1034600007F03CD00001230EC96F110ECA6F07ECA4
:1034700007F0010E3CEC07F02E0E88EC06F0000E73
:103480003CEC07F00001230EC96F130ECA6F07EC66
:1034900007F024D000019A0EC96F110ECA6F07EC15
:1034A00007F01CD000012C0EC96F120ECA6F07EC7A
:1034B00007F014D034CFE8FF000FF4E6B50FF2E7C1
:1034C0004B0F020D290EF324F66E100EF420F76E4A
:1034D0000900F5500900F5CFFAFFF96E320E000130
:1034E000BA6FBB6B14EC23F02C0E88EC06F02FCFD8
:1034F000E8FF3CEC07F02C0E88EC06F02ECFE8FF3E
:103500003CEC07F011840D0E88EC06F065EC07F03A
:1035100080920F01346B1200C696C694C682C69084
:1035200082840001BC6BBD6BFF0EDBEC23F000015D
:10353000BC4BBD2B000EBD5D0A0ED8B4BC5DD8A03F
:10354000F3D78294F36AF46AF34AF42AC30EF45C64
:10355000500ED8B4F35CD8A0F7D70001F66BF76B28
:10356000F86BF96B400E09DA22CA00F00004D8A407
:10357000000C0001F66BF76BF86BF96B770EFDD959
:1035800022CAE8FF050AD8A422D00001796B7A6B21
:10359000010EE8CF22FA0A012253D8B413D0000159
:1035A000F66BF76BF86BF96B410EE7D900017A51B6
:1035B000030AE80ED8B47919D8B4000C792B000EA0
:1035C0007A23E9D7C696C694C692C680010C00013C
:1035D000796B7A6B010EE8CF22FA0A012253D8B434
:1035E0001AD00001F66BF76BF86BF96B690EC5D951
:1035F0000001F66BF76BF86BF96B770EBED9000123
:103600007A51030AE80ED8B47919D8B4000C792B92
:10361000000E7A23E2D7C696C694C692C680010CE5
:10362000A7000001A76BA86BA96BAA6B4D0EB7D9B9
:10363000A7C0E1FFA8C0E2FF00EE01F0E150E926DB
:10364000E250EA2222CAEFFF23CAE7FF010CBC00C6
:103650000001796B7A6B010EE8CF22FA0A0122533E
:10366000D8B410D00001BE6BBF6BC06BC16B7A0EBB
:10367000ADD90001791D7A11D8B4000C792B000E58
:103680007A23ECD7BCC0E1FFBDC0E2FF00EE03F03F
:10369000E150E926E250EA2223CAEFFF00EE02F0F1
:1036A000E150E926E250EA2224CAEFFF00EE01F0E1
:1036B000E150E926E250EA2225CAEFFF26CAE7FFD9
:1036C000010CBC000001F66BF76BBCC0F8F0BDC08C
:1036D000F9F0500E52D90A012253D8A4000C010C63
:1036E000EC000001090ED890EC37ED37EE37EF37DC
:1036F000E82EF9D7EEC0F6FFEFC0F7FFECC0F3FFFE
:10370000EDC0F4FFF6CFF6F0F7CFF7F0F3CFF8F017
:10371000F4CFF9F0510E31D90A012253D8A4000C8C
:103720000001796B7A6BFF0EDBEC23F0FE0AD8B454
:1037300012D0000179C000F07AC001F00028796F42
:1037400002E101287A6F030E015CE80ED8B4005C38
:10375000D8B0000CE8D7F2C0E1FFF3C0E2FF006A86
:10376000016A026A036AC968C7A0FED70001F15165
:10377000F011D8A403D0C9CFE6FF06D0C9CFE7FF28
:103780000001F007D8A0F107002A000E0122022252
:103790000322035C08E1000E025C05E1020E015CFD
:1037A00002E1000E005CD8A0DED7FF0EDBEC23F0B8
:1037B000FF0EDBEC23F0010CCF000001090ED890C6
:1037C000CF37D037D137D237E82EF9D7D1C0F3FF72
:1037D000D2C0F4FFCFC0F6FFD0C0F7FFF3CFF6F0B2
:1037E000F4CFF7F0F6CFF8F0F7CFF9F0510EC5D8D7
:1037F0000A012253D8A4000C0001796B7A6BFF0EEA
:10380000DBEC23F0FE0AD8B412D0000179C000F03E
:103810007AC001F00028796F02E101287A6F030E67
:10382000015CE80ED8B4005CD8B0000CE8D7D3C077
:10383000E1FFD4C0E2FFD96AC968C7A0FED7C9CFEB
:10384000E6FFD92EF9D7C968C7A0FED7C9CFE6FFD2
:10385000D92EF9D7FF0EDBEC23F0FF0EDBEC23F0C3
:10386000010CA7000001090ED890A737A837A93787
:10387000AA37E82EF9D7A9C0F6FFAAC0F7FFA7C05C
:10388000F3FFA8C0F4FFF6CFF6F0F7CFF7F0F3CFD1
:10389000F8F0F4CFF9F0580E70D80A012253D8A4EA
:1038A000000CFF0EDBEC23F0FF0EDBEC23F0FE0E32
:1038B000DBEC23F00001A86BA96B0001A851AB253C
:1038C000E96EA951AC21EA6EEF50DBEC23F0000168
:1038D000A84BA92B020EA95D000ED8B4A85DD8A0F4
:1038E000ECD7FF0EDBEC23F0FF0EDBEC23F0FF0E3A
:1038F000DBEC23F00001A76FFF0EDBEC23F0006E82
:103900000028D8B4010CF8D7FB000001FF6F0A01B2
:10391000216BFF0EDBEC23F00001FF51DBEC23F009
:103920000001FF5178D80001FC51DBEC23F00001CD
:10393000FC5171D80001FB51DBEC23F00001FB517D
:103940006AD80001FE51DBEC23F00001FE5163D880
:103950000001FD51DBEC23F00001FD515CD80AEEC3
:1039600021F0D890EF360A01212B21CAE8FFDBECC9
:1039700023F0FF0EDBEF23F0F6000001FA6FF6C034
:10398000FBF0F7C0FCF0F8C0FDF0F9C0FEF0BDDFC1
:10399000FF0EDBEC23F0E8CF22FA1200A7000001B3
:1039A000A76FA7C0FBF0A8C0FCF0A9C0FDF0AAC09B
:1039B000FEF0ABDFFF0EDBEC23F0E8CF22FAFF0EC8
:1039C000DBEC23F0E8CF23FA1200BE000001C26F47
:1039D000BEC0FBF0BFC0FCF0C0C0FDF0C1C0FEF037
:1039E00094DFFF0EDBEC23F0E8CF22FAFF0EDBECD6
:1039F00023F0E8CF23FAFF0EDBEC23F0E8CF24FA24
:103A0000FF0EDBEC23F0E8CF25FAFF0EDBEC23F012
:103A1000E8CF26FA1200D96E080EE16E0AEE21F008
:103A2000D890EF360A01D9AE02D0090E211B21AF82
:103A300003D00A01090E211BD890D936E12EEED70A
:103A40001200EC00ECC0F6FFEDC0F7FF0F0EF764BC
:103A500003D00800F55005D0F6CFE9FFF7CFEAFF15
:103A6000EF501200DD000001E86BE96BDDC0E1FF03
:103A7000DEC0E2FF0001E151EC6FE251ED6FE14B7E
:103A8000E22BE0DF0001E76FE751D8B4E1D100019C
:103A9000E751250AD8B404D0E751E36FE7D9EAD754
:103AA0000001E469E66BE56B93D10001E051DF11A1
:103AB000D8B406D0DFC0E9FFE0C0EAFF000EEF6A2D
:103AC000E8C000F0E9C001F01200E1CFE9FFE2CF69
:103AD000EAFF020EE126000EE222EF500001B1D112
:103AE0000001E58D75D10001E52B0A0E04D0100E02
:103AF00001D0080E0001E46FE6CFF6FFE6CFF7FF36
:103B00000001E5A10DD0F7AE06D0F66CF71ED8B0D7
:103B1000F72AE60707D00001E591E5AD03D0F9D714
:103B20000001E591E4C002F0036AF6CF00F0F7CFA0
:103B300001F023EC24F000500001E76FE4C002F034
:103B4000036AF6CF00F0F7CF01F023EC24F004C0B5
:103B5000F6FF05C0F7FF010EEA6FEB6B0001EB51BA
:103B6000F75C02E1EA51F65CD8A010D0E4C002F0A4
:103B7000036AEAC000F0EBC001F084EC24F004C05A
:103B8000EAF005C0EBF00001E607E8D70001E5A97F
:103B900005D00BD0200E0001E36F68D90001E607C5
:103BA000E651800A7F0FD8B0F5D70001E5A104D017
:103BB0002D0EE36F5BD906D00001E5AD03D02B0ECF
:103BC000E36F54D90001E5B905D02ED0300E0001C5
:103BD000E36F4CD90001E607E651800A7F0FD8A0B9
:103BE00023D0F4D7EAC002F0EBC003F0F6CF00F028
:103BF000F7CF01F023EC24F004C000F005C001F081
:103C0000E4C002F0036A23EC24F000500001E66FE8
:103C1000E651800A760FD8A002D0070EE6270001F1
:103C2000E651300FE36F22D9E4C002F0036AEA0ED6
:103C3000E96E000EEA6EEE50006EEF50016E23EC5E
:103C400024F00550ED6E0450EF6EEE50ED10D8A448
:103C5000C9D7090E0001E76502D0070EE72700016A
:103C6000E751300FE36F02D905D70001E651800A12
:103C70007E0FD8A006D0200E0001E36FF7D8E6072C
:103C8000F4D7E1CFE9FFE2CFEAFF020EE126000E12
:103C9000E222EF500001E76FE751E36FE7D8EAD681
:103CA000E1CFE9FFE2CFEAFF020EE126000EE222B9
:103CB000EECF00F0EDCF01F000C077F001C078F05A
:103CC0000001E76B77C000F078C001F00001E75118
:103CD0000024026E000E0120036E02C0F6FF03C036
:103CE000F7FF0F0EF76403D00800F55005D0F6CFAC
:103CF000E9FFF7CFEAFFEF500009D8B403D0000185
:103D0000E72BE0D70001E451E76102D0E751E46F0F
:103D10000001E451E6BF1ED0FF0AE625D8A01AD064
:103D2000200E0001E36FA2D8E607F2D7000177C0AA
:103D300000F078C001F00028776F02E10128786F69
:103D400000C0ECF001C0EDF07DDE0001E76FE7514F
:103D5000E36F8CD80001E407E429D8B48BD6E6D70A
:103D6000E1C0ECF0E2C0EDF06DDE2A0AD8A40ED07E
:103D7000E1CFE9FFE2CFEAFF020EE126000EE222E8
:103D8000EF500001E46FE14BE22B22D00001E15142
:103D9000EC6FE251ED6FE14BE22B54DED00F0001EE
:103DA000E46FE1C0ECF0E2C0EDF04CDE0001E76F43
:103DB0002F0EE7650DD03A0EE7610AD0E4510A0DE7
:103DC000E751F324D00FDED70001E5B52DD0E5890A
:103DD0000001E151EC6FE251ED6FE14BE22B32DE7D
:103DE0000001E76FE75101E160D62A0A01E16DD6D3
:103DF000010A01E175D6050AB3E01E0AE5E0680A8A
:103E000001E175D63B0A01E130D7070A01E16BD623
:103E10000B0A01E16ED61C0A01E142D7060A01E154
:103E20006BD60D0A01E163D62F0E0001E7650BD0BA
:103E30003A0EE76108D0E585E6510A0DE751F32413
:103E4000D00FE66FC5D70001E751E36F0FD812D648
:103E50000001E051DF11D8B406D0DFC0E9FFE0C0B7
:103E6000EAFF000EEF6A0001E72B13D0E84BE92BC5
:103E7000E051DF11D8B409D0DFC0E9FFE0C0EAFFAC
:103E8000E3C0EFFFDF4BE02B12000001E351C0EF76
:103E900023F0E8C000F0E9C001F01200D96E11D0A3
:103EA000120EE8CF27FA010EE8CF28FA0ED00A0149
:103EB0002753D8A40AD028CA00F00028D8B4000C90
:103EC00004D0D950EDE0010AF2E000018F0EC96F75
:103ED000000ECA6F27CACBF028CACCF0CD6BCE6BD0
:103EE000010ECF6F4ED92CCA27FA2DCA28FA010C21
:103EF00000018F0EC96F000ECA6F120ECB6FCC6B14
:103F0000CD6BCE6B010ECF6F3CD9F66AF76A010E0E
:103F1000D96E11D0D950120AD8B40CD0D950040D92
:103F20002C0EF324E96E0A0EF420EA6EEF50F6260A
:103F3000000EF722D92A230ED964ECD7F6CF00F071
:103F4000F7CF01F01200BA000F01346B0001C26B11
:103F50000001C251A3DF0009D8B40ED1010E000147
:103F6000C26FF46A05D1F438E846E00B020FF36E35
:103F7000F3500AEE2CF0E926000EEA22EF50D8B4F6
:103F8000F6D0F3500AEE2CF0E926000EEA22EF50AC
:103F9000800AD8B4ECD0F3501AEE2DF0E126000ED2
:103FA000E222BCC0E9FFBDC0EAFFE7CFEFFFF3505C
:103FB0001AEE2EF0E126000EE222BEC0E9FFBFC0DD
:103FC000EAFFE7CFEFFFF3500AEE48F0E926000ED4
:103FD000EA22EF50006EF3500AEE49F0E926000E97
:103FE000EA22EF50036E00C002F0C0C0E9FFC1C07A
:103FF000EAFF02C0EEFF03C0EDFF020ED96ED92A20
:10400000D950130AD8B4010CD9500001BA25006E5A
:10401000000EBB21016EFD0E0024E96EFF0E012093
:10402000EA6EEF50D8B411D0F350D9CF00F0016A46
:104030000026000E01222C0E0024E96E0A0E01203B
:10404000EA6EEF50A00AD8B492D0D9500001BA2538
:10405000006E000EBB21016EFD0E0024E96EFF0E06
:104060000120EA6EEF50D8A411D0F350D9CF00F060
:10407000016A0026000E01222C0E0024E96E0A0EB1
:104080000120EA6EEF50A00AD8A471D0D9500001E7
:10409000BA25006E000EBB21016EFD0E0024E96EF4
:1040A000FF0E0120EA6EEF50D8A411D0F350D9CF03
:1040B00000F0016A0026000E01222C0E0024E96E99
:1040C0000A0E0120EA6EEF50A00AD8B4010CD950B4
:1040D0000001BA25006E000EBB21016EFD0E00240A
:1040E000E96EFF0E0120EA6EEF503F0AD8A40FD010
:1040F000F350D9CF00F0016A0026000E01222C0EE9
:104100000024E96E0A0E0120EA6E3F0EEF6ED950D0
:104110000001BA25006E000EBB21016EFD0E0024C9
:10412000E96EFF0E0120EA6EEF502A0AD8B4010CA6
:10413000D950BA25006E000EBB21016EFD0E002481
:10414000E96EFF0E0120EA6EEF50006EF350D9CFFA
:1041500002F0036A0226000E03222C0E0224E96EEE
:104160000A0E0320EA6EEF500018D8B448D7F42A9C
:10417000070EF464F8D6ECD63E0EE8CF34FF000C00
:10418000C900CBC02FFFCCC02EFF046A056A066AA7
:10419000076A0001CB07CB29D8B41CD0CBC000F0F4
:1041A000016A0050000FF66E0150F76E100EF722F4
:1041B0000800F550016E006A000E01BEFF0E026E8F
:1041C000036E0050042601500522025006220350BF
:1041D0000722DFD70001CC51016E006A000E01BE3C
:1041E000FF0E026E036E005004260150052202509D
:1041F000062203500722CD510426010ED8B0052611
:10420000D8B00626D8B00726C9C0D0F0CAC0D1F0B1
:1042100004C0D2F005C0D3F006C0D4F007C0D5F07A
:10422000CEC0D6F0CFC0D7F021EC04F0010C819CB9
:10423000819E818A81988194320EF0EC22F08184F3
:10424000819A210E48D8C50E46D8060E44D8130EC2
:1042500042D8200E40D80C0E3ED00001D76B000E85
:1042600030D80001F80EBA6F010EBB6F0001BA51D1
:10427000006EBB51016EBA07000EBB5B015000100F
:10428000D8B41200000E4DD8F1D70001D76B000E44
:1042900018D80001A76BA86B0001A805F80ED8B4C8
:1042A000A719D8B41200A74BA82BA751A90FF66ED7
:1042B000A851F76E180EF7220800F55032D8ECD747
:1042C000D7000001D86FD851060DF350800F03D8E6
:1042D0000001D751400FE96E8198E950E16E080E58
:1042E000D96ED950D8B41200819C020EE8CF29FAB9
:1042F0000A0100F000F0292F79EF21F0D906E1AE94
:1043000002D0818E01D0819E818C020EE8CF29FAE5
:104310000A0100F000F0292F89EF21F0D890E13652
:10432000E0D7E96E8188D9D712801200129012006E
:10433000006E0050050DF350A90FF66EF450F76EA5
:10434000130E12B045D0F7220800F550EADF0050F6
:10435000050DF350A90FF66EF450F76E130EF72209
:10436000F62A000EF7220800F550DBDF0050050D9D
:10437000F350A90FF66EF450F76E130EF722020EEB
:10438000F626000EF7220800F550CBDF0050050D91
:10439000F350A90FF66EF450F76E130EF722030ECA
:1043A000F626000EF7220800F550BBDF0050050D81
:1043B000F350A90FF66EF450F76E130EF722040EA9
:1043C000F626000EF7220800F550ABDF000EA9D745
:1043D000F7220800F550FE08A4DF0050050DF35049
:1043E000A90FF66EF450F76E130EF722F62A000EA0
:1043F000F7220800F550FE0894DF0050050DF35039
:10440000A90FF66EF450F76E130EF722020EF62681
:10441000000EF7220800F550FE0883DF0050050D5E
:10442000F350A90FF66EF450F76E130EF722030E39
:10443000F626000EF7220800F550FE0872DF005045
:10444000050DF350A90FF66EF450F76E130EF72218
:10445000040EF626000EF7220800F550FE0861DF74
:10446000FE0E5FD7D700D96ED7C002F0036AD950CD
:10447000520DF3CF00F0F4CF01F0D4EC07F004C0FC
:10448000F6FF05C0F7FF7E0E4CDF520EF36EF46AA6
:10449000F350006EF450016EF306000EF45A015012
:1044A0000010D8B411D0F750F45C02E1F650F35C80
:1044B000D8A004D00001D751D8A403D0420E31DFD8
:1044C000E7D77E0E2EDFE4D77E0E2BD7BA00000191
:1044D000BE51006EBF51016EBE07000EBF5B0150A2
:1044E0000010D8B45ED0BAC0F6FFBBC0F7FF0F0E05
:1044F000F76403D00800F55005D0F6CFE9FFF7CFF9
:10450000EAFFEF500009D8B422D0BCC0F6FFBDC00E
:10451000F7FF0F0EF76403D00800F55005D0F6CF73
:10452000E9FFF7CFEAFFEF50006EBAC0F6FFBBC05D
:10453000F7FF0F0EF76403D00800F55005D0F6CF53
:10454000E9FFF7CFEAFFEF500018D8B424D0BAC083
:10455000F6FFBBC0F7FF0F0EF76403D00800F5505D
:1045600005D0F6CFE9FFF7CFEAFFEF50006E016A02
:10457000BCC0F6FFBDC0F7FF0F0EF76403D0080004
:10458000F55005D0F6CFE9FFF7CFEAFFEF50005E18
:10459000000E015A12000001BA4BBB2BBC4BBD2BC5
:1045A00096D7006A016A1200CE000001CF51D96E81
:1045B0000BD0D906FD0EE8CF29FA0A0100F000F071
:1045C000292FDEEF22F00400010ED960F2D7CEC011
:1045D00029FA0A0100F000F0292FEAEF22F0120078
:1045E000E16E040ED96EFA0EE8CF29FA0A0100F046
:1045F00000F0292FF7EF22F00400D92EF4D7E12E96
:10460000F0D71200E16E040ED96EFA0EE8CF29FA47
:104610000A0100F000F0292F09EF23F0D92EF5D779
:10462000E12EF1D71200BA00040ED96EFA0EE8CFCF
:1046300029FA0A0100F000F0292F1AEF23F00400F4
:10464000D92EF4D7BA0EE96E000EEA6EEE06000E11
:10465000ED5AEE50ED10D8B41200E6D7F36E040E0A
:10466000E96EFA0EBDDF0400E92EFBD7F32EF7D773
:104670001200E96AEA6A0C6A086A096A0A6A0B6A3D
:10468000045005100610071006E1046A056A066A60
:10469000076AE9EF07F0C00E0C1606D0D890043672
:1046A0000536063607360C2A07AEF8D70C2AD890FE
:1046B000083609360A360B360750035C08E1065007
:1046C000025C05E10550015C02E10450005C09E375
:1046D00008800450005E0550015A0650025A0750E7
:1046E000035AD89007320632053204320C060C50B9
:1046F0003F0BDDE10CBCB3EC24F00050046E015024
:10470000056E0250066E0350076E0850006E095089
:10471000016E0A50026E0B50036E0CAEEDEF07F007
:10472000B3EC24F0EDEF07F00F0E806E816A440EBB
:10473000826E3D0E926E010E936E930E946E810EFC
:10474000C26E8E0EC16EC79EC79CC688C696C694A2
:10475000C682C690C68A810EAF6E240EAC6E900ED5
:10476000AB6EF28AD76AD66AD59CD59AD596D5848F
:10477000D582D580F19CF288D08EF28CF28E120018
:104780000001EC6F0AD0ACA2FED70001EC51AD6E77
:1047900012000001EC5198EF21F0000E11B0010E53
:1047A000026E036A05D00250EEE0010AF2E0120048
:1047B0000350F9E01200C96EC7A0FED7C95012001D
:1047C000E96AEA6A0050086E0150096E02500A6EEA
:1047D00003500B6E026A036A08500402F3CF00F024
:1047E000F4CF01F00502F3500126F45002220950E3
:1047F0000402F3500126F4500222D8B0032A0850D4
:104800000602F3500226F450032209500502F35029
:104810000226F45003220A500402F3500226F450F8
:10482000032208500702F350032609500602F350F2
:1048300003260A500502F35003260B500402F350DE
:104840000326EDEF07F0066A046A056A02500310BA
:1048500003E1006A016A000C1F0E0612D890062AB6
:1048600002360336FCE3033202320250005C03508E
:10487000015804E3016E0250005ED880043605360C
:10488000062E06BAF0D706AE05D0041E042AD8B408
:104890000506051E0450026E0550036E06AC000CA2
:1048A000001E002AD8B40106011E000C006E046A26
:1048B000D890FD0E01241AE3036AF00E011403E1FF
:1048C000040E036E013A026AD890032A0136FDE312
:1048D00001320150005CD8B0006E0236032EF8D7CA
:1048E00004BE026C025004BE006C1200013206E2EB
:1048F0000132D8A0006AD8900032D8A0D89000C069
:1049000002F0006A0036ECD702500002F3CF04F048
:10491000F4CF05F00102F350052603500002F350D6
:1049200005261200046E042A0406D8B4000CD890A0
:104930000036013602360336F7D7DFC0E1F0E0C0BB
:10494000E2F0000EE8CFDFF0E8CFE0F033EF1DF04B
:10495000046E042A0406D8B4000CD8900332023244
:1049600001320032F7D7001E011E021E031E000E88
:10497000002A0122022203221200EE6AEA50E262B9
:0A498000FCD7E950E162F9D71200FC
:00000001FF
